:020000040800F2
:100000000006022001020008B50F0008350F0008A5
:100010008D0F0008350F0008610F0008030200086B
:100020000302000803020008030200083928000840
:10003000030200080302000803020008030200088C
:10004000030200080302000803020008030200087C
:1000500003020008030200089D390008C5390008A2
:10006000ED390008153A00083D3A0008030200087F
:10007000030200080302000803020008030200084C
:10008000030200080302000803020008030200083C
:10009000030200080302000803020008653A000892
:1000A000030200080302000803020008030200081C
:1000B0004D3B000803020008030200080302000889
:1000C00003020008030200080302000803020008FC
:1000D00003020008030200080302000803020008EC
:1000E000C93A0008030200080302000803020008DE
:1000F00003020008030200080302000803020008CC
:1001000003020008030200080302000803020008BB
:1001100003020008030200080302000803020008AB
:10012000030200080302000803020008030200089B
:10013000030200080302000803020008030200088B
:10014000030200080302000803020008ED2F000864
:10015000030200080302000803020008030200086B
:10016000030200080302000803020008030200085B
:10017000030200080302000803020008030200084B
:100180000302000803020008393B000803020008CC
:10019000030200080302000803020008030200082B
:1001A000030200080302000803020008030200081B
:1001B000030200080302000803020008030200080B
:1001C00003020008030200080302000803020008FB
:1001D00003020008030200080302000803020008EB
:1001E00003020008030200080302000803020008DB
:1001F00003020008030200080302000803020008CB
:1002000002E000F000F8FEE772B63A4880F3088892
:10021000394880F3098839484EF60851CEF200017A
:10022000086040F20000CCF200004EF63471CEF2CD
:1002300000010860BFF34F8FBFF36F8F40F20000E3
:10024000C0F2F0004EF68851CEF200010860BFF314
:100250004F8FBFF36F8F4FF00000E1EE100A4EF6A4
:100260003C71CEF200010860062080F31488BFF3D1
:100270006F8F02F09FFB02F041FB03F031FA4FF069
:1002800055301F491B4A91423CBF41F8040BFAE725
:100290001C49194A91423CBF41F8040BFAE71A493C
:1002A0001A4A1B4B9A423EBF51F8040B42F8040B0A
:1002B000F8E700201749184A91423CBF41F8040B67
:1002C000FAE702F059FB03F06BFA144C144DAC4200
:1002D00003DA54F8041B8847F9E700F041F8114CA1
:1002E000114DAC4203DA54F8041B8847F9E702F0D9
:1002F00041BB00000006022000220220000000088E
:100300000000022000060220783F000800220220A0
:1003100068220220682202207834022000020008AD
:100320000002000800020008000200082DE9F04F5A
:100330002DED108AC1F80CD0D0F80CD0BDEC108A8D
:10034000BDE8F08F002383F311882846A0470020E2
:1003500001F07AFEFEE701F0F5FD00DFFEE70000A8
:1003600038B502F051FA40B1174B6FF07F0100220F
:1003700059720E211A729972DA7202F01BFA05464E
:1003800002F050FA0446D0B9104B9D4219D0013307
:100390009D4241F2883512BF044600250124002009
:1003A00002F012FA0CB100F079F800F06BFD00F0E9
:1003B0000DFC284600F0FCF800F070F8F9E7002585
:1003C000EDE70546EBE700BF00220220010007B081
:1003D00008B500F0C7FBA0F120035842584108BD02
:1003E00007B541F21203022101A8ADF8043000F074
:1003F000D7FB03B05DF804FB38B5202383F31188E5
:100400001748C3680BB101F0A5FE0023154A4FF44D
:100410007A71134801F062FE002383F31188124CB5
:10042000236813B12368013B2360636813B16368D9
:10043000013B63600D4D2B7833B963687BB90220B3
:1004400000F09AFC322363602B78032B07D163689A
:100450002BB9022000F090FC4FF47A73636038BD32
:1004600068220220F9030008842302207C22022053
:10047000084B187003280CD8DFE800F008050208C4
:10048000022000F06FBC022000F062BC024B002290
:100490005A6070477C22022084230220F8B53F4B2B
:1004A0003F4A1C461968013177D004339342F9D191
:1004B0006268A24271D33B4B9B6803F1006303F572
:1004C000C0339A4269D2002000F09AFB0220FFF765
:1004D000CFFF354B00211A6C19641A6E19661A6E1B
:1004E0005A6C59645A6E59665A6E5A6942F08002C3
:1004F0005A615A6922F080025A615A691A6942F0B7
:1005000000521A611A6922F000521A611B6972B610
:100510004FF0E023C3F8084DD4E90004BFF34F8F38
:10052000BFF36F8F214AC2F88410BFF34F8F536916
:1005300023F480335361BFF34F8FD2F8803043F6FA
:10054000E076C3F3C905C3F34E335B0103EA060C3F
:1005500029464CEA81770139C2F87472F9D2203BFE
:1005600013F1200FF2D1BFF34F8FBFF36F8FBFF3A3
:100570004F8FBFF36F8F536923F400335361002310
:10058000C2F85032BFF34F8FBFF36F8F202383F336
:100590001188854680F308882047F8BD008001084F
:1005A00020800108002202200038024000ED00E017
:1005B0002DE9F04F93B0B44B2022FF2100900AA800
:1005C0009D6800F009FCB14A1378A3B90121B04835
:1005D0001170C360202383F31188C3680BB101F04D
:1005E000B9FD0023AB4A4FF47A71A94801F076FDBA
:1005F000002383F31188009B13B1A74B009A1A6064
:10060000A64A1378032B03D000231370A24A536029
:100610004FF0000A009CD3465646D146012000F018
:10062000A1FB24B19C4B1B68002B00F0268200200C
:1006300000F098FA0390039B002BF2DB012000F0FE
:1006400087FB039B213B1F2BE8D801A252F823F024
:10065000D1060008F90600088D0700081D060008ED
:100660001D0600081D0600081F080008EF09000805
:10067000090900086B09000893090008B909000876
:100680001D060008CB0900081D0600083D0A0008E9
:10069000710700081D060008810A0008DD06000831
:1006A000710700081D0600086B0900081D060008F8
:1006B0001D0600081D0600081D0600081D0600088E
:1006C0001D0600081D0600081D0600088D0700080D
:1006D0000220FFF77DFE002840F0F981009B0221F7
:1006E00005A8BAF1000F08BF1C4641F21233ADF85D
:1006F000143000F055FA91E74FF47A7000F032FAB6
:10070000071EEBDB0220FFF763FE0028E6D0013F67
:10071000052F00F2DE81DFE807F0030A0D10133623
:100720000523042105A8059300F03AFA17E00421F7
:100730005548F9E704215A48F6E704215948F3E7F8
:100740004FF01C08404608F1040800F05BFA042151
:10075000059005A800F024FAB8F12C0FF2D1012081
:100760004FF0000900FA07F747EA0B0B5FFA8BFB23
:1007700000F07EFB26B10BF00B030B2B08BF00240F
:10078000FFF72EFE4AE704214748CDE7002EA5D00B
:100790000BF00B030B2BA1D10220FFF719FE07462C
:1007A00000289BD00120002600F02AFA0220FFF743
:1007B0005FFE5FFA86F8404600F032FA0446B0B1B8
:1007C000039940460136A1F140025142514100F0E7
:1007D00037FA0028EDD1BA46044641F2121302213D
:1007E00005A83E46ADF8143000F0DAF916E72546C4
:1007F0000120FFF73DFE244B9B68AB4207D92846FA
:1008000000F000FA013040F067810435F3E700257D
:10081000224BBA463E461D701F4B5D60A8E7002E76
:100820003FF45CAF0BF00B030B2B7FF457AF0220B0
:10083000FFF71EFE322000F095F9B0F10008FFF638
:100840004DAF18F003077FF449AF0F4A08EB0503DB
:10085000926893423FF642AFB8F5807F3FF73EAFD4
:10086000124BB845019323DD4FF47A7000F07AF90A
:100870000390039A002AFFF631AF039A0137019BD8
:1008800003F8012BEDE700BF0022022080230220A5
:1008900068220220F9030008842302207C2202201F
:1008A00004220220082202200C22022080220220A0
:1008B000C820FFF78DFD074600283FF40FAF1F2D1E
:1008C00011D8C5F120020AAB25F003008449424546
:1008D000184428BF4246019200F058FA019AFF21BD
:1008E0007F4800F079FA4FEAA803C8F387027C49F1
:1008F0002846019300F078FA064600283FF46DAFD1
:10090000019B05EB830533E70220FFF761FD00281B
:100910003FF4E4AE00F0C0F900283FF4DFAE00275A
:10092000B846704B9B68BB4218D91F2F11D80A9B41
:1009300001330ED027F0030312AA134453F8203CCE
:1009400005934046042205A9043700F035FB804694
:10095000E7E7384600F056F90590F2E7CDF8148045
:10096000042105A800F01CF902E70023642104A873
:10097000049300F00BF900287FF4B0AE0220FFF7DB
:1009800027FD00283FF4AAAE049800F06DF9059009
:10099000E6E70023642104A8049300F0F7F8002898
:1009A0007FF49CAE0220FFF713FD00283FF496AEC3
:1009B000049800F069F9EAE70220FFF709FD002832
:1009C0003FF48CAE00F078F9E1E70220FFF700FD7C
:1009D00000283FF483AE05A9142000F073F9074600
:1009E0000421049004A800F0DBF83946B9E732206E
:1009F00000F0B8F8071EFFF671AEBB077FF46EAECD
:100A0000384A07EB0903926893423FF667AE02202B
:100A1000FFF7DEFC00283FF461AE27F003074F44E8
:100A2000B9453FF4A5AE484609F1040900F0EAF8DB
:100A30000421059005A800F0B3F8F1E74FF47A70AF
:100A4000FFF7C6FC00283FF449AE00F025F9002866
:100A500044D00A9B01330BD008220AA9002000F0E1
:100A6000C3F900283AD02022FF210AA800F0B4F9E7
:100A7000FFF7B6FC1C4801F0EDFA13B0BDE8F08FAB
:100A8000002E3FF42BAE0BF00B030B2B7FF426AEA6
:100A90000023642105A8059300F078F80746002894
:100AA0007FF41CAE0220FFF793FC804600283FF441
:100AB00015AEFFF795FC41F2883001F0CBFA0598AE
:100AC00000F018FA46463C4600F0D2F9A6E5064684
:100AD0004EE64FF0000901E6BA467EE637467CE670
:100AE0008022022000220220A0860100F7B50C46D9
:100AF000184E4FF47A71054602FB01F396F9002077
:100B0000501C0BD11448294601930268176A2246EB
:100B1000B8478442019B03D1002310E0002AF1D0A2
:100B200096F90020511C01D0012A0DD10B4829460D
:100B30000268166A2246B047844205D10123084A5A
:100B40000120137003B0F0BD4FF4FA7001F082FA87
:100B50000020F7E710220220F8270220D4230220E9
:100B6000D0230220002307B5024601210DF1070022
:100B70008DF80730FFF7BAFF20B19DF8070003B0EA
:100B80005DF804FB4FF0FF30F9E700000A4604214E
:100B900008B5FFF7ABFF80F00100C0B2404208BDCE
:100BA000074B0A4630B41978064B53F821400146EA
:100BB00023682046DD69044BAC4630BC604700BF6B
:100BC000D0230220283C0008A086010070B50A4E00
:100BD00000240A4D01F0E0FC30802868338883420D
:100BE00008D901F0D3FC2B6804440133B4F5C03FAD
:100BF0002B60F2D370BD00BFD22302208C230220D1
:100C000001F08CBD00F1006000F5C0300068704755
:100C100000F10060920000F5C03001F00BBD000053
:100C2000054B1A68054B1B889B1A834202D9104456
:100C300001F0ACBC002070478C230220D22302209C
:100C400038B50446074D29B128682044BDE838402E
:100C500001F0BCBC2868204401F0A0FC0028F3D0BF
:100C600038BD00BF8C23022010F0030309D1B0F57A
:100C7000846F04D200F10050A0F57120036818467B
:100C800070470023FBE7000000F10050A0F5712041
:100C9000D0F8200470470000064991F8243033B1A1
:100CA00000230822086A81F82430FFF7B1BF012031
:100CB000704700BF90230220014B1868704700BFA7
:100CC000002004E0204B0246F0B518681F4BC0F32B
:100CD0000B06000C1F885D68BE4293F9084022D0C5
:100CE0009F89BE4221D01F8BBE4206D102240C2513
:100CF00005FB04335D6893F90840B0F5805F16D0BA
:100D000041F20103984208BF5A24013A013D0B46C3
:100D10000A4493420DD215F9016F581C5EB1034687
:100D200000F8016CF5E70024E1E70124DFE7412446
:100D3000EBE7184605E02C2590421D7001D2981C67
:100D40005C70401AF0BD00BF002004E014220220B5
:100D5000022803D1024B4FF080629A61704700BFB6
:100D6000000C0240022803D1024B4FF480629A61CA
:100D7000704700BF000C0240022804D1024A5369A8
:100D800083F4806353617047000C0240002310B568
:100D9000934203D0CC5CC4540133F9E710BD00008A
:100DA000013810B510F9013F3BB191F900409C4268
:100DB00003D11AB10131013AF4E71AB191F90020D7
:100DC000981A10BD1046FCE703460246D01A12F9E5
:100DD000011B0029FAD1704702440346934202D016
:100DE00003F8011BFAE770472DE9F8431F4D14463D
:100DF0000746884695F8242052BBDFF870909CB3D4
:100E000095F824302BB92022FF2148462F62FFF7A6
:100E1000E3FF95F824004146C0F1080205EB80008D
:100E2000A24228BF2246D6B29200FFF7AFFF95F844
:100E30002430A41B17441E449044E4B2F6B2082E9A
:100E400085F82460DBD1FFF727FF0028D7D108E021
:100E50002B6A03EB82038342CFD0FFF71DFF0028EC
:100E6000CBD10020BDE8F8830120FBE790230220CE
:100E7000024B1A78024B1A70704700BFD023022031
:100E80001022022038B5154C154D204600F0F0FB1D
:100E90002946204600F018FC2D681248EA6ED2F868
:100EA000043843F00203C2F8043801F0D3F80E49C5
:100EB000284600F011FDEA6E0C48D2F804380C49BF
:100EC000A04223F00203C2F804384FF4E1330B6070
:100ED00003D0BDE8384000F02BBB38BDF827022016
:100EE000343D000840420F003C3D0008D42302205E
:100EF000B823022038B50B4B04461A780A4B53F836
:100F000022500A4B9D420CD0094B00211822184652
:100F1000FFF762FF046001462846BDE8384000F054
:100F200007BB38BDD0230220283C0008F827022048
:100F3000B823022000B59BB0EFF309816822684610
:100F4000FFF724FFEFF30583044B9A6BDA6A9A6A82
:100F50009A6A9A6A9A6A9A6A9B6AFEE700ED00E0CA
:100F600000B59BB0EFF3098168226846FFF70EFFDA
:100F7000EFF30583044B9A6B9A6A9A6A9A6A9A6AA3
:100F80009A6A9B6AFEE700BF00ED00E000B59BB0E7
:100F9000EFF3098168226846FFF7F8FEEFF3058357
:100FA000034B5A6B9A6A9A6A9A6A9A6A9B6AFEE734
:100FB00000ED00E0FEE7000030B50A44084D914224
:100FC0000DD011F8013B5840082340F30004013BC9
:100FD0002C4013F0FF0384EA5000F6D1EFE730BD58
:100FE0002083B8ED026843681143016003B11847DC
:100FF00070470000024A136843F0C0031360704753
:101000000078004013B50E4C204600F085FA04F13C
:10101000140000234FF480720A49009400F046F94E
:10102000094B4FF48072094904F13800009400F034
:10103000BFF9074A074BC4E9172302B010BD00BF30
:10104000D423022040240220F50F0008402502206E
:101050000078004080F93703037C30B5214C00292B
:1010600018BF0C46012B0CD11F4B984209D11F4BC6
:101070001A6C42F080421A641A6E42F080421A667C
:101080001B6E2268036EC16D03EB52038466B3FBD3
:10109000F2F36268150442BF23F0070503F007036B
:1010A00043EA4503CB60A36843F040034B60E36829
:1010B00043F001038B6042F4967343F001030B602D
:1010C0004FF0FF330B62510505D512F0102205D009
:1010D000B2F1805F04D080F8643030BD7F23FAE73E
:1010E0003F23F8E7303C0008D423022000380240B8
:1010F0002DE9F047C66D05463768F469210734626B
:1011000019D014F0080118BF8021E20748BF41F050
:101110002001A3074FF0200348BF41F040016007C2
:1011200048BF41F4807183F31188281DFFF75AFFEF
:10113000002383F31188E2050AD5202383F3118865
:101140004FF40071281DFFF74DFF002383F3118832
:101150004FF020094FF0000A14F0200838D13B0668
:1011600016D54FF0200905F1380A200610D589F36D
:101170001188504600F050F9002836DA0821281D61
:10118000FFF730FF27F080033360002383F31188DB
:10119000790614D5620612D5202383F31188D5E988
:1011A00013239A4208D12B6C33B127F0400710214A
:1011B000281DFFF717FF3760002383F31188E3062C
:1011C00018D5AA6E1369ABB15069BDE8F04718474E
:1011D00089F31188736A284695F86410194000F065
:1011E000B5F98AF31188F469B6E7B06288F311881B
:1011F000F469BAE7BDE8F087F8B515468268044699
:101200000B46AA4200D28568A1692669761AB542C2
:101210000BD218462A46FFF7B9FDA3692B44A361F8
:101220002846A3685B1BA360F8BD0CD9AF1B18460A
:101230003246FFF7ABFD3A46E1683044FFF7A6FDC2
:10124000E3683B44EBE718462A46FFF79FFDE36857
:10125000E5E7000083689342F7B50446154600D2DF
:101260008568D4E90460361AB5420BD22A46FFF7E6
:101270008DFD63692B4463612846A3685B1BA360F3
:1012800003B0F0BD0DD93246AF1B0191FFF77EFDD3
:1012900001993A46E0683144FFF778FDE3683B4442
:1012A000E9E72A46FFF772FDE368E4E710B50A4470
:1012B0000024C361029B8460C16002610362C0E9D3
:1012C0000000C0E9051110BD08B5D0E90532934210
:1012D00001D1826882B98268013282605A1C4261FF
:1012E00019700021D0E904329A4224BFC3684361D7
:1012F00000F0CCFE002008BD4FF0FF30FBE70000FF
:1013000070B5202304460E4683F31188A568A5B165
:10131000A368A269013BA360531CA36115782269ED
:10132000934224BFE368A361E3690BB12046984769
:10133000002383F31188284607E03146204600F059
:1013400095FE0028E2DA85F3118870BD2DE9F74F8C
:1013500004460E4617469846D0F81C904FF0200AD7
:101360008AF311884FF0000B154665B12A463146C5
:101370002046FFF741FF034660B94146204600F092
:1013800075FE0028F1D0002383F31188781B03B089
:10139000BDE8F08FB9F1000F03D001902046C84797
:1013A000019B8BF31188ED1A1E448AF31188DCE748
:1013B000C160C361009B82600362C0E905111144F2
:1013C000C0E9000001617047F8B504460D461646B5
:1013D000202383F31188A768A7B1A368013BA3600A
:1013E00063695A1C62611D70D4E904329A4224BFB9
:1013F000E3686361E3690BB120469847002080F3FE
:10140000118807E03146204600F030FE0028E2DA7D
:1014100087F31188F8BD0000D0E9052310B59A4282
:1014200001D182687AB982680021013282605A1C37
:1014300082611C7803699A4224BFC368836100F00B
:1014400025FE204610BD4FF0FF30FBE72DE9F74F9A
:1014500004460E4617469846D0F81C904FF0200AD6
:101460008AF311884FF0000B154665B12A463146C4
:101470002046FFF7EFFE034660B94146204600F0E4
:10148000F5FD0028F1D0002383F31188781B03B009
:10149000BDE8F08FB9F1000F03D001902046C84796
:1014A000019B8BF31188ED1A1E448AF31188DCE747
:1014B000026843681143016003B118477047000098
:1014C0001430FFF743BF00004FF0FF331430FFF735
:1014D0003DBF00003830FFF7B9BF00004FF0FF33C9
:1014E0003830FFF7B3BF00001430FFF709BF00002A
:1014F0004FF0FF311430FFF703BF00003830FFF723
:1015000063BF00004FF0FF323830FFF75DBF0000CF
:1015100000207047FFF776BD044B03600023436053
:10152000C0E9023301230374704700BF483C000840
:1015300010B52023044683F31188FFF78DFD0223A5
:101540002374002383F3118810BD000038B5C369EC
:1015500004460D461BB904210844FFF7A9FF29469C
:1015600004F11400FFF7B0FE002806DA201D4FF446
:101570008061BDE83840FFF79BBF38BD0268436813
:101580001143016003B118477047000013B5446B65
:10159000D4F8A4381A681178042915D1217C0229BD
:1015A00012D11979012312898B4013420CD101A960
:1015B00004F14C0001F09AFFD4F8A4480246019BC4
:1015C0002179206800F0D4F902B010BD143001F088
:1015D0001DBF00004FF0FF33143001F017BF0000B3
:1015E0004C3001F0EFBF00004FF0FF334C3001F002
:1015F000E9BF0000143001F0EBBE00004FF0FF31F6
:10160000143001F0E5BE00004C3001F0BBBF00001B
:101610004FF0FF324C3001F0B5BF000000207047A2
:10162000D0F8A4381A6810B511780446042917D1E7
:10163000017C022914D15979012352898B4013422C
:101640000ED1143001F07EFE024648B1D4F8A44811
:101650004FF4807361792068BDE8104000F076B9DE
:1016600010BD0000406BFFF7DBBF000070470000BB
:101670007FB5124B01250426044603600023057440
:1016800000F1840243602946C0E902330C4B02900A
:10169000143001934FF48073009601F02FFE094B34
:1016A00004F29442294604F14C000294CDE900630F
:1016B0004FF4807301F0F6FE04B070BD703C00087A
:1016C000651600088D1500080B68202282F311882A
:1016D0000A7903EB820210624A790D3243F8220044
:1016E0008A7912B103EB820318620223C0F8A418AE
:1016F0000374002383F311887047000038B5037F1B
:10170000044613B190F85430ABB90125201D0221D5
:10171000FFF734FF04F114006FF00101257700F0AA
:10172000C1FC04F14C0084F854506FF00101BDE895
:10173000384000F0B7BC38BD10B501210446043074
:10174000FFF71CFF0023237784F8543010BD0000FE
:1017500038B504460025143001F0E8FD04F14C00D2
:10176000257701F0B7FE201D84F854500121FFF7C2
:1017700005FF2046BDE83840FFF752BF90F85C30C7
:1017800003F06003202B06D190F85D200023212A6E
:1017900003D81F2A06D800207047222AFBD1C0E9AF
:1017A000143303E0034A0265072242658365012082
:1017B000704700BF38220220D0F8A43837B51A6825
:1017C0000446117804291AD1017C022917D119790C
:1017D000012312898B40134211D100F14C05284698
:1017E00001F038FF58B101A9284601F07FFED4F876
:1017F000A4480246019B2179206800F0B9F803B0A3
:1018000030BD000000EB8103F0B51E6A85B00446D0
:101810000D46FEB1202383F3118804EB8507301DAC
:101820000821FFF7ABFEFB6806F14C005B691B6803
:101830001BB1019001F068FE019803A901F056FE6A
:10184000024648B1039B2946204600F091F8002348
:1018500083F3118805B0F0BDFB685A691268002A4D
:10186000F5D01B8A013B1340F1D104F15C02EAE799
:101870000D3138B550F82140DCB1202383F31188B5
:10188000D4F8A4281368527903EB8203DB689B69C0
:101890005D6845B104216018FFF770FE294604F128
:1018A000140001F059FD2046FFF7BAFE002383F330
:1018B000118838BD7047000001F0F2B801232822DA
:1018C000002110B5044600F8243BFFF785FA0023F9
:1018D000C4E9013310BD000038B50446202383F36A
:1018E000118800254160C0E90355C0E90555C0E9EC
:1018F000075501F0E5F80223237085F3118838BD00
:1019000070B500EB8103054650690E461446DA6057
:1019100018B110220021FFF75FFAA06918B1102258
:101920000021FFF759FA31462846BDE8704001F022
:1019300091B90000826802F0011282600022C0E9C1
:101940000422C0E90622026201F010BAF0B40125B7
:1019500000EB810447898D40E4683D43A4694581DB
:1019600023600023A2606360F0BC01F02BBA00008A
:10197000F0B4012500EB810407898D40E4683D4304
:101980006469058123600023A2606360F0BC01F0FC
:10199000A5BA000070B50223002504460370456611
:1019A000056280F84C50C0E90255C0E90455C0E911
:1019B000065501F0EBF863681B6823B12946204601
:1019C000BDE87040184770BD037880F86830052383
:1019D000037043681B6810B504460BB10421984797
:1019E0000023A36010BD000090F8682043680270D7
:1019F0001B680BB1052118477047000070B590F8BF
:101A00004C30044613B1002380F84C3004F15C02E2
:101A1000204601F0CDF963689B68B3B994F85C3057
:101A200013F0600535D00021204601F033FC002181
:101A3000204601F025FC63681B6813B1062120468F
:101A40009847062384F84C3070BD204698470028FC
:101A5000E4D0B4F86230626D9A4288BF636594F94D
:101A60005C30656D002B4FF0200380F20381002D68
:101A700000F0F280092284F84C2083F311880021C1
:101A80002046D4E91423FFF773FF002383F3118862
:101A9000DAE794F85D2003F07F0343EA022340F283
:101AA0000232934200F0C58021D8B3F5807F48D040
:101AB0000DD8012B3FD0022B00F09380002BB2D128
:101AC00004F16402226502226265A365C1E7B3F5F1
:101AD000817F00F09B80B3F5407FA4D194F85E3005
:101AE000012BA0D1B4F8643043F0020332E0B3F527
:101AF000006F4DD017D8B3F5A06F31D0A3F5C063F8
:101B0000012B90D86368204694F85E205E6894F8B4
:101B10005F10B4F86030B047002884D04368236574
:101B2000036863651AE0B3F5106F36D040F60242E1
:101B300093427FF478AF5C4B2365022363650023F7
:101B4000C3E794F85E30012B7FF46DAFB4F86430D6
:101B500023F00203A4F86430C4E91455A56578E7BE
:101B6000B4F85C30B3F5A06F0ED194F85E30204627
:101B700084F8663001F062F863681B6813B10121D4
:101B800020469847032323700023C4E914339CE7BD
:101B900004F1670323650123C3E72378042B10D1E5
:101BA000202383F311882046FFF7C4FE85F31188B4
:101BB0000321636884F8675021701B680BB12046CD
:101BC000984794F85E30002BDED084F86730042309
:101BD000237063681B68002BD6D0022120469847EB
:101BE000D2E794F8603020461D0603F00F010AD5B5
:101BF00001F0D0F8012804D002287FF414AF2B4B59
:101C00009AE72B4B98E701F0B7F8F3E794F85E30CA
:101C1000002B7FF408AF94F8603013F00F01B3D0BD
:101C20001A06204602D501F049FBADE701F03CFB66
:101C3000AAE794F85E30002B7FF4F5AE94F860309C
:101C400013F00F01A0D01B06204602D501F022FBA5
:101C50009AE701F015FB97E7142284F84C2083F3F0
:101C600011882B462A4629462046FFF76FFE85F34A
:101C70001188E9E65DB1152284F84C2083F31188C0
:101C800000212046D4E91423FFF760FEFDE60B2275
:101C900084F84C2083F311882B462A462946204697
:101CA000FFF766FEE3E700BFA03C0008983C000891
:101CB0009C3C000838B590F84C300446002B3ED0D0
:101CC000063BDAB20F2A34D80F2B32D8DFE803F004
:101CD0003731310822323131313131313131373719
:101CE000456DB0F862309D4214D2C3681B8AB5FBC3
:101CF000F3F203FB12556DB9202383F311882B46B1
:101D00002A462946FFF734FE85F311880A2384F812
:101D10004C300EE0142384F84C30202383F31188D8
:101D2000002320461A461946FFF710FE002383F3CE
:101D3000118838BD836D03B198470023E7E7002180
:101D4000204601F0A7FA0021204601F099FA6368C5
:101D50001B6813B10621204698470623D7E70000E9
:101D600010B590F84C300446142B29D017D8062B08
:101D700005D001D81BB110BD093B022BFBD80021B7
:101D8000204601F087FA0021204601F079FA6368C5
:101D90001B6813B1062120469847062319E0152B2E
:101DA000E9D10B2380F84C30202383F311880023E2
:101DB0001A461946FFF7DCFD002383F31188DAE7A2
:101DC000C3689B695B68002BD5D1836D03B19847CD
:101DD000002384F84C30CEE7024B0022C3E90033E5
:101DE0009A60704740260220002382680374054BE6
:101DF0001B6899689142FBD25A6803604260106088
:101E0000586070474026022008B5202383F31188CC
:101E1000037C032B05D0042B0DD02BB983F3118841
:101E200008BD436900221A604FF0FF334361FFF79A
:101E3000DBFF0023F2E7D0E9003213605A60F3E7DA
:101E4000002382680374054B1B6899689142FBD894
:101E50005A68036042601060586070474026022054
:101E6000054B196908741868026853601A60186194
:101E700001230374FEF75ABA402602204B1C30B5EA
:101E8000044687B00A4D10D02B6901A8094A00F01A
:101E900025F92046FFF7E4FF049B13B101A800F0E9
:101EA00059F92B69586907B030BDFFF7D9FFF8E73A
:101EB00040260220091E000838B50C4D0446416139
:101EC0002B6981689A68914203D8BDE83840FFF7D2
:101ED0008BBF1846FFF7B4FF01232C610146237422
:101EE0002046BDE83840FEF721BA00BF4026022058
:101EF000044B1A681B6990689B68984294BF002045
:101F0000012070474026022010B5084C2368206944
:101F10001A6854602260012223611A74FFF790FF4F
:101F200001462069BDE81040FEF700BA40260220B5
:101F300008B5FFF7DDFF18B1BDE80840FFF7E4BFC3
:101F400008BD0000FFF7E0BFFEE7000010B50C4C35
:101F5000FFF742FF00F0B4F880220A49204600F063
:101F60003BF8012344F8180C037400F075FC0023BF
:101F700083F3118862B60448BDE8104000F04CB805
:101F800068260220A43C0008B43C000800F01CB9FC
:101F9000EFF3118020B9EFF30583202282F311883B
:101FA0007047000010B530B9EFF30584C4F308049E
:101FB00014B180F3118810BDFFF7BAFF84F31188C4
:101FC000F9E70000034A516853685B1A9842FBD84E
:101FD000704700BF001000E082600222028270475A
:101FE0008368A3F17C0243F80C2C026943F83C2C73
:101FF000426943F8382C074A43F81C2CC268A3F105
:10200000180043F8102C022203F8082C002203F8D1
:10201000072C70474503000810B5202383F311886F
:10202000FFF7DEFF00210446FFF746FF002383F39E
:102030001188204610BD0000024B1B6958610F201B
:10204000FFF70EBF40260220202383F31188FFF7FD
:10205000F3BF000008B50146202383F31188082050
:10206000FFF70CFF002383F3118808BD49B1064B2D
:1020700042681B6918605A60136043600420FFF7D0
:10208000FDBE4FF0FF3070474026022003689842A3
:1020900006D01A680260506018465961FFF7A4BE66
:1020A0007047000038B504460D462068844200D1D0
:1020B00038BD036823605C604561FFF795FEF4E777
:1020C000054B4FF0FF3103F11402C3E90522002252
:1020D000C3E90712704700BF4026022070B51C4EAE
:1020E00005460C46C0E9032301F0E6FA334653F8EF
:1020F000142F9A420DD130620A2C2CBF00190A30DD
:102100002A60C5E90124C6E90555BDE8704001F023
:10211000C1BA316A431AE31838BF1C469368A34218
:1021200002D9081901F0C4FA73699A6894420CD86C
:102130005A68AC602B606A6015609A685D60121B1B
:102140009A604FF0FF33F36170BDA41A1B68ECE78F
:102150004026022038B51B4C636998420DD0816837
:10216000D0E9003213605A600022C2609A680A44C3
:102170009A604FF0FF33E36138BD036822460021C7
:1021800042F8143F93425A60C16003D1BDE8384021
:1021900001F088BA9A688168256A0A449A6001F059
:1021A0008BFA6369411B9A688A42E5D9AB181D1AFC
:1021B000206A092D98BF01F10A02BDE83840104499
:1021C00001F076BA402602202DE9F041184C002794
:1021D00004F11406656901F06FFA236AAA68C11A4E
:1021E0008A4215D81344D5F80C802362D5E9003211
:1021F00013605A606369EF60B34201D101F052FA93
:1022000087F311882869C047202383F31188E1E709
:102210006169B14209D013441B1ABDE8F0410A2B91
:102220002CBFC0180A3001F043BABDE8F08100BFEE
:102230004026022000207047FEE7000070470000A3
:102240004FF0FF307047000002290CD0032904D062
:102250000129074818BF00207047032A05D8054800
:1022600000EBC2007047044870470020704700BF71
:10227000983D0008482202204C3D000870B59AB0F5
:1022800005460846144601A900F0C2F801A8FEF769
:102290009BFD431C0022C6B25B001046C5E900341A
:1022A00023700323023404F8013C01ABD1B20234A1
:1022B0008E4201D81AB070BD13F8011B013204F828
:1022C000010C04F8021CF1E708B5202383F3118800
:1022D0000348FFF771FA002383F3118808BD00BF9C
:1022E000F827022090F85C3003F01F02012A07D182
:1022F00090F85D200B2A03D10023C0E9143315E0C8
:1023000003F06003202B08D1B0F860302BB990F8AF
:102310005D20212A03D81F2A04D8FFF72FBA222ACA
:10232000EBD0FAE7034A0265072242658365012084
:10233000704700BF3F22022007B5052917D8DFE804
:1023400001F0191603191920202383F31188104A6C
:1023500001210190FFF7D4FA019802210D4AFFF7FD
:10236000CFFA0D48FFF7F4F9002383F3118803B087
:102370005DF804FB202383F311880748FFF7BEF9BB
:10238000F2E7202383F311880348FFF7D5F9EBE741
:10239000EC3C0008103D0008F827022038B50C4D31
:1023A0000C4C2A460C4904F10800FFF767FF05F1C1
:1023B000CA0204F110000949FFF760FF05F5CA726F
:1023C00004F118000649BDE83840FFF757BF00BFC9
:1023D000D030022048220220CC3C0008D63C000825
:1023E000E13C000870B5044608460D46FEF7ECFCDB
:1023F000C6B22046013403780BB9184670BD324688
:102400002946FEF7CDFC0028F3D10120F6E70000B5
:102410002DE9F84F05460C46FEF7D6FC2C49C6B20E
:102420002846FFF7DFFF08B10536F6B229492846EE
:10243000FFF7D8FF08B11036F6B2632E0DD8DFF8DB
:102440009080DFF89090244FDFF894A0DFF894B0EC
:102450002E7846B92670BDE8F88F29462046BDE89B
:10246000F84F01F0C3BB252E2ED107224146284646
:10247000FEF796FC70B9DBF8003007350C3444F8F1
:102480000C3CDBF8043044F8083CDBF8083044F836
:10249000043CDDE7082249462846FEF781FC98B94E
:1024A000A21C0E4B197802320909C95D02F8041CFE
:1024B00013F8011B01F00F015345C95D02F8031C1D
:1024C000F0D118340835C3E7013504F8016BBFE7D4
:1024D000B83D0008E13C0008CD3D000820F4F01FA5
:1024E0002CF4F01FC03D0008BFF34F8F024AD368A1
:1024F000DB03FCD4704700BF003C024008B5074B2B
:102500001B7853B9FFF7F0FF054B1A69002A04DA6C
:10251000044A5A6002F188325A6008BD2E33022004
:10252000003C02402301674508B5054B1B7833B9D1
:10253000FFF7DAFF034A136943F00043136108BD54
:102540002E330220003C02400B28F0B516D80C4C6C
:102550000C4923787BB90E460B4D0C234FF00062DB
:10256000013B55F8047B46F8042B13F0FF033A4473
:10257000F6D10123237051F82000F0BD0020FCE7C4
:102580006033022030330220E03D0008014B53F855
:1025900020007047E03D00080C2070470B2810B564
:1025A000044601D9002010BDFFF7CEFF064B53F8BB
:1025B00024301844C21A0BB90120F4E71268013222
:1025C000F0D1043BF6E700BFE03D00080B2838B52A
:1025D000044628D8FFF7DCFC0546FFF785FF2046B8
:1025E000FFF78CFF114AF323D360E300DBB243F41F
:1025F000007343F002031361136943F480331361E2
:10260000FFF772FFFFF7A0FF094B53F8241000F00B
:10261000E9F82846FFF788FFFFF7C4FC2046BDE82D
:102620003840FFF7BBBF002038BD00BF003C024070
:10263000E03D000812F001032DE9F04105460E4689
:1026400014464BD18218B2F1026F61D8314B1B682E
:1026500013F001035CD0FFF79BFC2F4FFFF74EFFF9
:10266000F323314640F20128FB60FFF73DFF032CC6
:1026700018D824F001046D1A274E40F201180C44BA
:10268000A14205EB010733692AD123F0010333612D
:10269000FFF74AFFFFF786FC0120BDE8F081043C0C
:1026A0000435E4E7AB07E4D13B6923F440733B61B5
:1026B0003B6943EA08033B6151F8046B2E60BFF3AA
:1026C0004F8FFFF711FF2B689E42E8D03B6923F044
:1026D00001033B61FFF728FFFFF764FC0020DCE704
:1026E00023F440733361336943EA080333610B8891
:1026F0003B80BFF34F8FFFF7F7FE3F88BFB231F843
:10270000023BBB42BCD0336923F001033361E1E7F4
:102710001846C2E700380240003C0240084908B5AC
:102720000B7828B11BB9FFF7E9FE01230B7008BD38
:10273000002BFCD00870BDE80840FFF7F5BE00BFD5
:102740002E3302200244074BD2B210B5904200D182
:1027500010BD441C00B253F8200041F8040BE0B255
:10276000F4E700BF502800400F4B30B51C6F240425
:1027700007D41C6F44F400741C671C6F44F40044BD
:102780001C670A4C02442368D2B243F4807323606E
:10279000074B904200D130BD441C51F8045B00B29D
:1027A00043F82050E0B2F4E70038024000700040E7
:1027B0005028004007B5012201A90020FFF7C2FF01
:1027C000019803B05DF804FB13B50446FFF7F2FF70
:1027D000A04205D0012201A900200194FFF7C4FF07
:1027E00002B010BD0144BFF34F8F064B884204D3A3
:1027F000BFF34F8FBFF36F8F7047C3F85C02203079
:10280000F4E700BF00ED00E000207047034B1A68BA
:102810001AB9034AD2F874281A6070476433022048
:102820000030024008B5FFF7F1FF024B1868C0F313
:10283000407008BD64330220EFF309830549683313
:102840004A6B22F001024A6383F30988002383F371
:102850001188704700EF00E0202080F3118862B6F5
:102860000D4B0E4AD96821F4E0610904090C0A43B2
:102870000B49DA60D3F8FC2042F08072C3F8FC20E8
:10288000084AC2F8B01F116841F00101116010221E
:10289000DA7783F82200704700ED00E00003FA05C4
:1028A00055CEACC5001000E0202310B583F311888D
:1028B0000E4B5B6813F4006314D0F1EE103AEFF3A3
:1028C00009844FF08073683CE361094BDB6B23663E
:1028D00084F30988FFF70CFB10B1064BA36110BD10
:1028E000054BFBE783F31188F9E700BF00ED00E03B
:1028F00000EF00E0570300085A03000870B5BFF36B
:102900004F8FBFF36F8F1A4A0021C2F85012BFF3E6
:102910004F8FBFF36F8F536943F400335361BFF39D
:102920004F8FBFF36F8FC2F88410BFF34F8FD2F871
:10293000803043F6E074C3F3C900C3F34E335B0148
:1029400003EA0406014646EA81750139C2F860527D
:10295000F9D2203B13F1200FF2D1BFF34F8F53690F
:1029600043F480335361BFF34F8FBFF36F8F70BD5C
:1029700000ED00E0FEE700000A4B0B480B4A9042D6
:102980000BD30B4BC11EDA1C121A22F003028B422E
:1029900038BF00220021FEF71FBA53F8041B40F88D
:1029A000041BECE7E03F0008783402207834022072
:1029B000783402207047000070B5D0E91B43002234
:1029C0004FF0FF359E6804EB42135101D3F8000924
:1029D000002805DAD3F8000940F08040C3F8000968
:1029E000D3F8000B002805DAD3F8000B40F0804044
:1029F000C3F8000B013263189642C3F80859C3F8B4
:102A0000085BE0D24FF00113C4F81C3870BD000021
:102A10001D4B03EB8002D2F80CC02DE9F043DCF82B
:102A20001420461CDD6ED2F800E005EB063605EBFF
:102A30004018516871450AD30122D5F8343802FA9A
:102A400000F023EA0000C5F83408BDE8F083AEEBDF
:102A50000103BCF81040A34228BF2346D8F8184908
:102A6000A4B2B3EB840FF0D89468A4F1040959F828
:102A7000047F3760A4EB09071F44042FF7D81C44D8
:102A80000B4494605360D4E768330220890141F01D
:102A90002001016103699B06FCD41220FFF792BA62
:102AA00010B5054C2046FEF709FF4FF0A043E36642
:102AB000024B236710BD00BF68330220343E00087C
:102AC00070B503780546012B50D12A4BC46E98424D
:102AD0001BD1294B0E2143205A6B42F080025A63CE
:102AE0005A6D42F080025A655A6D5A6942F080026E
:102AF0005A615A6922F080025A615B6900F0E8FB72
:102B00001E4BE3601E4BC4F800380023EE6EC4F881
:102B1000003EC02323604FF40413A3633369002BEA
:102B2000FCDA01230C203361FFF74CFA3369DB0731
:102B3000FCD41220FFF746FA3369002BFCDA00269A
:102B40002846A660FFF738FF6B68C4F81068DB689A
:102B5000C4F81468C4F81C684BB90A4BA3614FF061
:102B6000FF336361A36843F00103A36070BD064BAC
:102B7000F4E700BF683302200038024040140040F0
:102B800003002002003C30C0083C30C0F8B5C46EE1
:102B9000054600214FF000662046FFF777FF296FBA
:102BA00000234FF001128F684FF0FF30C4F8343823
:102BB000C4F81C2804EB431201339F42C2F8006999
:102BC000C2F8006BC2F80809C2F8080BF2D20B6811
:102BD000EA6E6B67636210231361166916F01006C4
:102BE000FBD11220FFF7EEF9D4F8003823F4FE638E
:102BF000C4F80038A36943F4402343F01003A361F1
:102C00000923C4F81038C4F814380A4BEB604FF0AD
:102C1000C043C4F8103B084BC4F8003BC4F810692B
:102C2000C4F800396B6F03F1100243F480136A6734
:102C3000A362F8BD103E000840800010C26E90F8FC
:102C40006610D2F8003823F4FE6343EA0113C2F899
:102C5000003870472DE9F84300EB8103C56E0C4640
:102C60008046DA680FFA81F94801166806F0030613
:102C7000731E022B05EB41134FF0000194BFB60405
:102C8000384EC3F8101B4FF0010104F1100398BF38
:102C900006F1805601FA03F3916998BF06F50046E4
:102CA00000293AD0578A04F15801374349016F503F
:102CB000D5F81C180B430021C5F81C382B18012728
:102CC000C3F81019A7405369611E9BB3138A928BF6
:102CD0009B08012A88BF5343D8F87420981842EA09
:102CE000034301F140022146C8F87400284605EB71
:102CF00082025360FFF7CAFE08EB8900C3681B8A93
:102D000043EA845348341E4364012E51D5F81C38DD
:102D10001F43C5F81C78BDE8F88305EB4917D7F8C1
:102D2000001B21F40041C7F8001BD5F81C1821EA4C
:102D30000303C0E704F13F030B4A2846214605EB95
:102D400083035A60FFF7A2FE05EB4910D0F8003963
:102D500023F40043C0F80039D5F81C3823EA0707EC
:102D6000D7E700BF0080001000040002026F126865
:102D70004267FFF721BE00005831C36E49015B581E
:102D800013F4004004D013F4001F0CBF02200120F4
:102D9000704700004831C36E49015B5813F400408E
:102DA00004D013F4001F0CBF022001207047000064
:102DB00000EB8101CB68196A0B6813604B685360A4
:102DC0007047000000EB810330B5DD68AA69136825
:102DD000D36019B9402B84BF402313606B8A1468F9
:102DE000C26E1C4402EB4110013C09B2B4FBF3F487
:102DF0006343033323F0030343EAC44343F0C04374
:102E0000C0F8103B2B6803F00303012B0ED1D2F85E
:102E1000083802EB411013F4807FD0F8003B14BF58
:102E200043F0805343F00053C0F8003B02EB4112E3
:102E3000D2F8003B43F00443C2F8003B30BD000031
:102E40002DE9F041244D0446EE6E06EB4013D3F815
:102E5000087B3807C3F8087B0AD5D6F81438190759
:102E600006D505EB840321462846DB685B68984756
:102E7000FA071FD5D6F81438DB071BD505EB8403FA
:102E8000D968CCB98B69488A5A68B2FBF0F600FB66
:102E900016228AB91868DA6890420DD2121AC3E96C
:102EA0000024202383F311880B482146FFF78AFF73
:102EB00084F31188BDE8F081012303FA04F26B89E1
:102EC00023EA02036B81CB68002BF3D02146024832
:102ED000BDE8F041184700BF6833022000EB8103D2
:102EE0004A0170B5DD68C36E6C692668E66056BB42
:102EF0001A444FF40020C2F810092A6802F00302B5
:102F0000012A0AB20ED1D3F8080803EB421410F4D8
:102F1000807FD4F8000914BF40F0805040F000508A
:102F2000C4F8000903EB4212D2F8000940F0044053
:102F3000C2F800090122D3F8340802FA01F1014372
:102F4000C3F8341870BD19B9402E84BF40202060EA
:102F500020681A442E8A8419013CB4FBF6F440EA36
:102F6000C44040F00050C6E7F8B504461E48C56EA0
:102F700005EB4413D3F80869F107C3F8086917D5BE
:102F8000D5F81038DA0713D500EB8403D9684B69FC
:102F90001F68DA68974218D2D21B00271A605F6058
:102FA000202383F311882146FFF798FF87F31188C8
:102FB000330617D50123D5F83428A340134211D086
:102FC0002046BDE8F840FFF723BD012303FA04F2D1
:102FD000038923EA020303818B68002BE8D0214692
:102FE0009847E5E7F8BD00BF683302202DE9F74FA9
:102FF000A24CE66E7569B3691D4015F48058756181
:1030000007D02046FEF7C6FC03B0BDE8F04FFFF73F
:103010004BBC002D12DAD6F8003E9F0705D0D6F83B
:10302000003E23F00303C6F8003ED6F80438934868
:1030300023F00103C6F80438FEF7D6FC280505D5B1
:103040008E48FFF7B9FC8D48FEF7BEFCA9040CD5ED
:10305000D6F8083813F0060FF36823F470530CBF4A
:1030600043F4105343F4A053F3602A0704D5636874
:10307000DB680BB181489847EB0200F18A80AF0210
:1030800027D5D4F86C9000274FF0010ADFF8ECB197
:1030900009EB4712D2F8003B03F44023B3F5802F2D
:1030A00011D1D2F8003B002B0DDA62890AFA07F33E
:1030B00022EA0303638104EB8703DB68DB6813B157
:1030C0003946584698470137236FFFB29B689F42A5
:1030D000DED9E80618D5E76E3A6AC2F30A1002F0A4
:1030E0000F0302F4F012B2F5802F00F09C80B2F5CD
:1030F000402F09D104EB8303002207F58057DB68DA
:103100001B6A904240F082802B03D6F818481DD5E8
:10311000E70302D50020FFF793FEA60302D50120A6
:10312000FFF78EFE600302D50220FFF789FE210320
:1031300002D50320FFF784FEE20202D50420FFF748
:103140007FFEA30202D50520FFF77AFE6F037FF50D
:103150005BAFE60702D50020FFF706FFA50702D503
:103160000120FFF701FF600702D50220FFF7FCFEF8
:10317000210702D50320FFF7F7FEE20602D504205F
:10318000FFF7F2FEA3067FF53FAF0520FFF7ECFE49
:103190003AE7E36E00274FF0010ADFF8E0B0019351
:1031A000236F5FFA87F99B6899453FF668AF019BEB
:1031B00003EB4913D3F8002902F44022B2F5802F23
:1031C00022D1D3F80029002A1EDAD3F8002942F0D0
:1031D0009042C3F80029D3F80029002AFBDB4946B6
:1031E000E06EFFF753FC22890AFA09F322EA03038F
:1031F000238104EB8903DB689B6813B14946584679
:1032000098474846FFF704FC0137C9E7910701D109
:10321000D7F80080072A02F101029CBF03F8018B56
:103220004FEA18286DE7023307F5805704EB830255
:103230005268D2F818C0DCF80820DCE9001CA1EBC9
:103240000C0C002188420AD104EB830463689B695B
:103250009A6802449A605A6802445A6054E711F02E
:10326000030F01D1D7F800808C4501F1010184BF23
:1032700002F8018B4FEA1828E4E700BF6833022008
:10328000C36E03EB4111D1F8003B43F40013C1F8C6
:10329000003B7047C36E03EB4111D1F8003943F492
:1032A0000013C1F800397047C36E03EB4111D1F828
:1032B000003B23F40013C1F8003B7047C36E03EBDF
:1032C0004111D1F8003923F40013C1F800397047D7
:1032D000090100F16043012203F56143C9B283F89B
:1032E000001300F01F039A4043099B0003F1604361
:1032F00003F56143C3F880211A60704730B5043389
:10330000039C0172002104FB0325C160C0E9065340
:10331000049B0363059BC0E90000C0E90422C0E9E7
:103320000842C0E90A11436330BD00000022416A2F
:10333000C260C0E90411C0E90A226FF00101FEF782
:10334000B1BE0000D0E90432934201D1C2680AB98B
:10335000181D704700207047036919600021C2687A
:103360000132C260C269134482699342036124BF7F
:10337000436A0361FEF78ABE38B504460D46E3682A
:103380003BB162690020131D1268A3621344E3621B
:1033900007E0237A33B929462046FEF767FE002866
:1033A000EDDA38BD6FF00100FBE70000C368C269C9
:1033B000013BC3604369134482699342436124BF64
:1033C000436A436100238362036B03B1184770476C
:1033D00070B52023044683F31188866A3EB9FFF74F
:1033E000CBFF054618B186F31188284670BDA36A45
:1033F000E26A13F8015B9342A36202D32046FFF70F
:10340000D5FF002383F31188EFE700002DE9F84F83
:1034100004460E46174698464FF0200989F3118856
:103420000025AA46D4F828B0BBF1000F09D14146C7
:103430002046FFF7A1FF20B18BF311882846BDE895
:10344000F88FD4E90A12A7EB050B521A934528BF4F
:103450009346BBF1400F1BD9334601F1400251F8AE
:10346000040B914243F8040BF9D1A36A403640356E
:103470004033A362D4E90A239A4202D32046FFF7DD
:1034800095FF8AF31188BD42D8D289F31188C9E724
:1034900030465A46FDF77AFCA36A5E445D445B44BD
:1034A000A362E7E710B5029C0433017204FB032119
:1034B000C460C0E906130023C0E90A33039B036319
:1034C000049BC0E90000C0E90422C0E9084243634C
:1034D00010BD0000026A6FF00101C260426AC0E9DB
:1034E00004220022C0E90A22FEF7DCBDD0E9042351
:1034F0009A4201D1C26822B9184650F8043B0B60C9
:103500007047002070470000C3680021C269013382
:10351000C3604369134482699342436124BF436A91
:103520004361FEF7B3BD000038B504460D46E368BD
:103530003BB1236900201A1DA262E2691344E362D1
:1035400007E0237A33B929462046FEF78FFD00288D
:10355000EDDA38BD6FF00100FBE700000369196088
:10356000C268013AC260C26913448269934203612E
:1035700024BF436A036100238362036B03B11847CE
:103580007047000070B520230D460446114683F3B2
:103590001188866A2EB9FFF7C7FF10B186F311882C
:1035A00070BDA36A1D70A36AE26A01339342A362ED
:1035B00004D3E16920460439FFF7D0FF002080F3EF
:1035C0001188EDE72DE9F84F04460D4690469946DF
:1035D0004FF0200A8AF311880026B346A76A4FB934
:1035E00049462046FFF7A0FF20B187F311883046F7
:1035F000BDE8F88FD4E90A073A1AA8EB0607974204
:1036000028BF1746402F1BD905F1400355F8042B5E
:103610009D4240F8042BF9D1A36A40364033A3629F
:10362000D4E90A239A4204D3E16920460439FFF71A
:1036300095FF8BF311884645D9D28AF31188CDE7DF
:1036400029463A46FDF7A2FBA36A3D443E443B446B
:10365000A362E5E7D0E904239A4217D1C3689BB17E
:10366000836A8BB1043B9B1A0ED01360C368013B85
:10367000C360C3691A4483699A42026124BF436AE2
:103680000361002383620123184670470023FBE790
:1036900000F094B84FF08043002258631A61022270
:1036A000DA6070474FF080430022DA607047000014
:1036B0004FF08043586370474FF08043586A70471B
:1036C0004B6843608B688360CB68C3600B69436160
:1036D0004B6903628B6943620B68036070470000AB
:1036E00008B52C4B40F2FF712B481A690A431A6146
:1036F0001A6922F4FF6222F007021A611A691A6B32
:103700000A431A631A6D0A431A65244A1B6D11464F
:10371000FFF7D6FF00F5806002F11C01FFF7D0FF34
:1037200000F5806002F13801FFF7CAFF00F5806004
:1037300002F15401FFF7C4FF00F5806002F170014F
:10374000FFF7BEFF00F5806002F18C01FFF7B8FFC4
:1037500000F5806002F1A801FFF7B2FF00F580607C
:1037600002F1C401FFF7ACFF00F5806002F1E00157
:10377000FFF7A6FF00F5806002F1FC01FFF7A0FF54
:1037800002F58C7100F58060FFF79AFFBDE80840F4
:1037900000F08AB80038024000000240403E0008B5
:1037A00008B500F003FAFEF7D1FBFFF72FF8BDE8EC
:1037B0000840FEF7F3BD0000704700000F4B1A6C85
:1037C00042F001021A641A6E42F001021A660C4AB3
:1037D0001B6E936843F0010393604FF080436B22AC
:1037E0009A624FF0FF32DA6200229A615A63DA601D
:1037F0005A6001225A611A60704700BF00380240C7
:10380000002004E04FF0804208B51169D3680B40F6
:10381000D9B29B076FEA0101116107D5202383F319
:103820001188FEF7B3FB002383F3118808BD000065
:103830001B4B4FF0FF3000211A696FEA42526FEACA
:1038400052521A611A69C2F30A021A611A695A6954
:1038500058615A6959615A691A6A62F080521A624B
:103860001A6A02F080521A621A6A5A6A58625A6ACE
:1038700059625A6A0B4A106840F480701060186FE1
:1038800000F44070B0F5007F03D04FF4803018672B
:103890001967536823F40073536000F05FB900BFE9
:1038A0000038024000700040364B4FF44041364A29
:1038B0001A64364A11601A6842F001021A601A68E6
:1038C0009207FCD59A6822F003029A602D4B9A6801
:1038D00012F00C02FBD1196801F0F90119609A602D
:1038E0001A6842F480321A601A689003FCD55A6F45
:1038F00042F001025A67234B5A6F9107FCD5244AC4
:103900005A601A6842F080721A60204B5A6852045A
:10391000FCD51A6842F480321A605A68D003FCD58C
:103920001A6842F400321A60184A53689903FCD5A9
:10393000144B1A689201FCD5164A9A6040F20112A3
:10394000C3F88C200022C3F8902040F20733124ABB
:103950001360136803F00F03072BFAD1094B9A6821
:1039600042F002029A609A6802F00C02082AFAD128
:103970005A6C42F480425A645A6E42F480425A664B
:103980005B6E704700380240000400100070004079
:10399000086C400900948838003C0240074A08B58A
:1039A000536903F00103536123B1054A13680BB156
:1039B00050689847BDE80840FEF776BF003C0140DC
:1039C000F8330220074A08B5536903F00203536134
:1039D00023B1054A93680BB1D0689847BDE8084009
:1039E000FEF762BF003C0140F8330220074A08B5E9
:1039F000536903F00403536123B1054A13690BB102
:103A000050699847BDE80840FEF74EBF003C0140B2
:103A1000F8330220074A08B5536903F008035361DD
:103A200023B1054A93690BB1D0699847BDE80840B6
:103A3000FEF73ABF003C0140F8330220074A08B5C0
:103A4000536903F01003536123B1054A136A0BB1A4
:103A5000506A9847BDE80840FEF726BF003C014089
:103A6000F8330220164B10B55C6904F478725A6181
:103A7000A30604D5134A936A0BB1D06A984760062F
:103A800004D5104A136B0BB1506B9847210604D52F
:103A90000C4A936B0BB1D06B9847E20504D5094AE9
:103AA000136C0BB1506C9847A30504D5054A936C71
:103AB0000BB1D06C9847BDE81040FEF7F5BE00BFD3
:103AC000003C0140F8330220194B10B55C6904F446
:103AD0007C425A61620504D5164A136D0BB1506DD4
:103AE0009847230504D5134A936D0BB1D06D9847C1
:103AF000E00404D50F4A136E0BB1506E9847A10431
:103B000004D50C4A936E0BB1D06E9847620404D56D
:103B1000084A136F0BB1506F9847230404D5054A28
:103B2000936F0BB1D06F9847BDE81040FEF7BCBE55
:103B3000003C0140F833022008B50348FDF7D8FAED
:103B4000BDE80840FEF7B0BED423022008B5FFF759
:103B500059FEBDE80840FEF7A7BE0000062108B5E3
:103B60000846FFF7B5FB06210720FFF7B1FB06214A
:103B70000820FFF7ADFB06210920FFF7A9FB06216E
:103B80000A20FFF7A5FB06211720FFF7A1FB06215E
:103B90002820FFF79DFB07211C20FFF799FB0C2134
:103BA0005220BDE80840FFF793BB000008B5FFF7BF
:103BB0003FFE00F00DF8FDF7ADFCFDF77DFEFDF7D3
:103BC00055FDFFF7F9FDBDE80840FFF761BD0000B6
:103BD0000023054A19460133102BC2E9001102F1F6
:103BE0000802F8D1704700BFF8330220034611F8ED
:103BF000012B03F8012B002AF9D1704753544D33A0
:103C000032463F3F3F3F3F3F0053544D33324637EC
:103C10005B347C355D780053544D333246375B3628
:103C20007C375D7800000000F8270220D4230220B2
:103C300000960000000000000000000000000000EE
:103C4000000000000000000000000000DD1400087B
:103C5000C914000805150008F1140008FD14000837
:103C6000E9140008D5140008C11400081115000853
:103C700000000000E9150008D5150008111600081D
:103C8000FD15000809160008F5150008E1150008E3
:103C9000CD1500081D1600080000000001000000FE
:103CA000000000006D61696E0000000069646C65D1
:103CB00000000000AC3C000880260220F82702200B
:103CC00001000000491F00080000000041726475F7
:103CD00050696C6F740025424F415244252D424C6F
:103CE000002553455249414C2500000002000000C8
:103CF000000000000518000871180008400040008E
:103D0000A0300220B03002200200000000000000BD
:103D10000300000000000000B518000800000000CB
:103D200010000000C0300220000000000100000070
:103D3000000000006833022001010200392300085E
:103D400049220008E5220008C922000843000000BB
:103D5000543D000809024300020100C0320904007A
:103D600000010202010005240010010524010001E8
:103D7000042402020524060001070582030800FF4F
:103D800009040100020A00000007050102400000CA
:103D9000070581024000000012000000A03D00085D
:103DA00012011001020000400912415700020102F5
:103DB000030100000403090425424F415244250039
:103DC0004D6174656B463736352D534500303132C1
:103DD00033343536373839414243444546000000D4
:103DE00000800000008000000080000000800000D3
:103DF00000000200000004000000040000000400B5
:103E000000000400000004000000040000000400A2
:103E100000000000FD190008B51C0008611D000825
:103E200040004000E0330220E033022001000000A7
:103E3000F033022080000000400100000500000077
:103E40000000802A00000000AAAAAAAA00000024FC
:103E5000FFFF00000000000000A00A0000000001B9
:103E600000000000AAAAAAAA00000001FFFF0000AB
:103E70000000000000000000000100000000000041
:103E8000AAAAAAAA00010000FFFF0000000000008B
:103E9000000000000040100000000000AAAAAAAA2A
:103EA00000400000FFFB00000000000000000000D8
:103EB0000081420000000000AAAAAAAA0040410016
:103EC000EFFF00000000008008000000000000007C
:103ED00000000000AAAAAAAA00000000FFFF00003C
:103EE00000000000000000000000000000000000D2
:103EF000AAAAAAAA00000000FFFF0000000000001C
:103F0000000000000000000000000000AAAAAAAA09
:103F100000000000FFFF00000000000000000000A3
:103F20000000000000000000AAAAAAAA00000000E9
:103F3000FFFF000000000000000000000000000083
:103F40000000000000000000000000000000000071
:103F50000000000000000000000000000000000061
:103F60000000000000000000000000000000000051
:103F700000000000000000008F00000000000000B2
:103F800000801E0000000000FF0000000000000094
:103F9000FC3B00083F00000049040000093C000809
:103FA0003F00000051040000173C00083F000000E3
:103FB00000960000000008009600000000080000C5
:103FC00004000000B43D00080000000000000000F4
:103FD00000000000000000000000000000000000E1
:00000001FF
